:020000040000FA
:1000000065EF0CF01200FFFFFFFFFFFFFFFFFFFF98
:1008000065EF0CF01200FFFFFFFFFFFFFFFFFFFF90
:10081000FFFFFFFFFFFFFFFFFFFFFFFFFFFFFFFFE8
:10082000FFFFFFFFFFFFFFFFFFFF0100EC180000CD
:100830002201000002000000040120511F0B0108EA
:1008400001E05BD02051600BE842E842E842E84218
:10085000E842010801E051D0245103E0240501E001
:100860004CD02151230A48E0010A40E0030A30E05D
:10087000010A25E0240A22E0070A1FE0010A1CE021
:10088000030A11E0010A01E038D00101030E176FDD
:100890000101F50E186F000E196F01011F93010180
:1008A000080E1C6F2AD00101030E176F0101F50E0F
:1008B0001A6F000E1B6F21D020D01FD01ED0010157
:1008C000030E176F0101EA0E1A6F000E1B6F15D091
:1008D0000101030E176F0101EA0E186F000E196F68
:1008E00001011F930101070E1C6F07D00101030EC8
:1008F000176F22C4F1F001D000D012000001EA6BA2
:10090000C20EEB6F010EEC6FED6BEE6BEF6B080E32
:10091000F06FE36BE26B1A0E726E1E0E736E0401C3
:10092000000E166F050E176F400E146F0401196F3D
:10093000080E1A6F050E1B6F880E186F0401480E03
:100940001E6F050E1F6F400E1C6F1200D9CFE6FF01
:10095000E1CFD9FF0001E26B040118BF30D0FC0EDB
:10096000DBCF10F01951D880105403E2FC0E19C4EB
:10097000DBFF0001E26BFC0EDB50E25D19E2E251AD
:10098000EA6A080FE96E050EEA22EF50E66EE251C0
:10099000E76EFD0EDBCFE9FFFE0EDBCFEAFFE7508F
:1009A000E926000EEA22E552E750EF6EE22BE3D78C
:1009B0000401400E196F1817187D880E18130001D6
:1009C000E25100D0E552E7CFD9FF1200D9CFE6FFC0
:1009D000E1CFD9FFE6520001E35101E02FD0DF6AF9
:1009E000DF2ADF50106E116AFF0E101801E111505E
:1009F00001E10BD0FD0EDBCFE9FFDB2AFE0EDBCFE2
:100A0000EAFF01E3DB2AEF50EBE1DF50106E116AE1
:100A1000D950FD0FE96EFF0EDA20EA6E1050EE5E3F
:100A20001150ED5AFD0EDBCFE4F0FE0EDBCFE5F00A
:100A3000DFCFE8F00001E96B010EE36FE552E5520C
:100A4000E7CFD9FF1200D9CFE6FFE1CFD9FFE652B9
:100A50000001E35101E030D0DF6ADF2ADF50106E81
:100A6000116AFF0E101801E1115001E10CD0FD0ECA
:100A7000DBCFF6FFDB2AFE0EDBCFF7FF01E3DB2A3D
:100A80000800F550EAE1DF50106E116AD950FD0FF1
:100A9000E96EFF0EDA20EA6E1050EE5E1150ED5A4C
:100AA000FD0EDBCFE4F0FE0EDBCFE5F0DFCFE8F0AC
:100AB0000001010EE96FE36FE552E552E7CFD9FF80
:100AC0001200D9CFE6FFE1CFD9FFE65204011CBFE7
:100AD0006BD0030E0001E35D01E1E36BE35101E143
:100AE00063D0020EE35D06E104011D6B0001030EFD
:100AF000E36F54D0E30552E1400E106E116AE851E5
:100B0000105C000E115803E2400EDF6E02D0E8C008
:100B1000DFFFDFCF1DF4DF50E85DE86F480EE66FC2
:100B2000050EE76FE90515E1DF5012E0E4C0F6FFBE
:100B3000E5C0F7FF0800F550E6C0E9FFE7C0EAFFAF
:100B4000EF6EE62B000EE723E42BE523DF06ECD760
:100B500013D0DF5011E0E4C0E9FFE5C0EAFFEF5039
:100B6000E6C0E9FFE7C0EAFFEF6EE62B000EE723E1
:100B7000E42BE523DF06EDD7E85110E104011D5118
:100B8000106E116A400E101801E1115004E10001CD
:100B9000020EE36F03D00001030EE36F400E040169
:100BA0001C171C7D880E1C13E552E552E7CFD9FFB8
:100BB000120004012051600BE842E842E842E8429A
:100BC000E842000901E055D02151070A51E00B0A23
:100BD0004FE0070A40E0010A2CE00B0A28E0020A75
:100BE00026E0030A22E0080A12E0010A0EE00F0ADA
:100BF0000AE0030A01E03CD00101010E176F010178
:100C0000040E1E6F36D036D834D090D832D00101C1
:100C1000010E176F0101200E186F010E196F0101EF
:100C20001F930101010E1C6F24D0A8D822D0F6D842
:100C300020D00101010E176F040124510101186F2A
:100C4000196B210E1827010E192301011F930101B1
:100C5000010E1C6F0ED00101010E176F040124510B
:100C6000EA6A210FE96E010EEA2222C4EFFF01D0E9
:100C700000D01200800E0401205D57E12351030AC9
:100C800034E0010A10E0030A01E04DD00101010E39
:100C9000176F01013C0E186F160E196F120E01012D
:100CA0001C6F1D6B40D00101010E176F0401225112
:100CB000F66EF76AD890F636F736FD0EF626160E63
:100CC000F7220900F5CF18F10A00F5CF19F1020E4D
:100CD0000101F76A1825F66E1951F7220900F5CFC0
:100CE0001CF10A00F5CF1DF11ED00101010E176F96
:100CF00004012251F66EF76AD890F636F736010EE7
:100D0000F626170EF7220900F5CF18F10A00F5CFE5
:100D100019F118C1F6FF19C1F7FF0800F5500101DC
:100D20001C6F1D6B00D001011F8312000101010E19
:100D3000176F0F0EE66E710EE66E0F0EE66E56EC36
:100D40000AF0E552E552E552010EE66E210EE66E1E
:100D5000010EE66E56EC0AF0E552E552E55222C469
:100D600020F10401225104E10101050E1E6F05D09E
:100D70000101060E1E6F7EEC04F012000401286BC8
:100D8000296B040120511F0B020A16E0030A10E030
:100D9000010A01E035D00101010E176F80A402D0D5
:100DA0000401288101011FA102D00401288328D059
:100DB0000101010E176F24D00101010E176F04010C
:100DC00024510F0B080DF350116A000F106E040E22
:100DD00011222451800B01E0010E040DF35001019A
:100DE00010241A6F000E11201B6F1AC1E9FF1BC1DE
:100DF000EAFFEF50040B03E00401010E286F00D05E
:100E0000010117050AE10101280E186F040E196F80
:100E100001011F930101020E1C6F12000401220543
:100E200010E120511F0B00090CE10101010E176FA9
:100E3000030E0401215D03E101011F8102D00101C4
:100E40001F91040122513AE120511F0B020836E1A3
:100E500024510F0B000932E00101010E176F04014C
:100E600024510F0B080DF350116A000F106E040E81
:100E700011222451800B01E0010E040DF3500101F9
:100E800010241A6F000E11201B6F030E0401215D48
:100E900007E1840E1AC1E9FF1BC1EAFFEF6E0ED015
:100EA00024AF06D01AC1E9FF1BC1EAFFEF6A06D0E2
:100EB000880E1AC1E9FF1BC1EAFFEF6E12006C50E9
:100EC00002E0000E01D0010E00090BE00401005108
:100ED0003C0BE842E8420D0802E10CD801D040D8B2
:100EE00008D06C5002E0000E01D0010E040901E0B0
:100EF00047D81200D9CFE6FFE1CFD9FFE652010172
:100F0000166B176B1C6B1D6BD9EC05F0DF6ADF509D
:100F1000106E116A010E105C000E11581BE20101E7
:100F2000175101E017D0F76ADF34FE0BF736F66E83
:100F3000070EF626170EF7220900F5CF10F008006D
:100F4000F5CF11F004D011C0FAFF1050F96EFBDF9D
:100F5000DF2ADDD7DDD8E552E552E7CFD9FF120011
:100F6000020E0101165D0AE196D8040100BD03D00E
:100F7000C80E006F02D0880E006F01D00FD912008A
:100F8000040E01011E5D0AE122C46EFF6E500008CE
:100F900003E2050E1E6F02D0030E1E6F010116053F
:100FA0000AE10BD8040104BD03D0C80E046F02D0BF
:100FB000880E046F01D0F2D81200D9CFE6FFE1CF3E
:100FC000D9FF020EE1260101080E1C5D000E1D591D
:100FD00005E21CC1DEFF1DC1DDFF03D0080EDE6E81
:100FE000DD6A040104930491010EDB500413DFCF8A
:100FF00005F4000EDB5001011C5F010EDB501D5B90
:10100000280E1A6F040E1B6F01011FA31ED0D9CF2B
:10101000E9FFDACFEAFFEE50ED1016E018C1F6FF57
:1010200019C1F7FF0800F5501AC1E9FF1BC1EAFF1B
:10103000EF6E01011A2B000E1B23182B1923DF065C
:10104000010E01E2DB06E3D71CD0D9CFE9FFDACFEE
:10105000EAFFEE50ED1015E018C1E9FF19C1EAFFF3
:10106000EF501AC1E9FF1BC1EAFFEF6E01011A2B15
:10107000000E1B23182B1923DF06010E01E2DB06ED
:10108000E4D7020EE15C02E2E16AE552E16EE5526C
:10109000E7CFD9FF1200D9CFE6FFE1CFD9FF020E8B
:1010A000E126030E04010015E76E010EE7CFDBFF1A
:1010B00001C4DFFFDE5001011C27DD501D23280E77
:1010C000186F040E196FD9CFE9FFDACFEAFFEE509F
:1010D000ED1014E018C1E9FF19C1EAFFEF501AC181
:1010E000E9FF1BC1EAFFEF6E1A2B000E1B23182B22
:1010F0001923DF06010E01E2DB06E5D7020EE15CF3
:1011000002E2E16AE552E16EE552E7CFD9FF120053
:10111000010117510CE10401080E016F200E026F4E
:10112000040E036F840E006F0401046F35D00401B8
:1011300020AF22D001011C510401265D01011D5187
:101140000401275904E226C41CF127C41DF135DF30
:101150000101010E166F0401080E016F200E026FCF
:10116000040E036F800E006F0401280E066F040E3C
:10117000076FC80E046F10D00101020E166F040134
:10118000056BC80E046F0401080E016F280E026F74
:10119000040E036FC80E006F6D9812000101166BEC
:1011A0000401080E016F200E026F040E036F880EFB
:1011B000006F0401046B12008A849394E66A030EA4
:1011C000E66E020EE66ED4EC0BF0E552E552E55207
:1011D0000101870E006F0C0E016F00EF09F08A9479
:1011E00071EC0CF00101016F71EC0CF00101006F6A
:1011F0008A8400B502D0000E02D0010E00D0120089
:10120000D9CFE6FFE1CFD9FF030EE12600C110F0F0
:1012100001C111F0D89011321032E804FBE110C086
:10122000DEFF11C0DDFFD950010FE96EDACFEAFF12
:10123000EF50100B08E1010EDB9ADB9CDB9E0101F5
:101240002B0E026F16D0010EDB8ADB8CDB8E0101C8
:101250002D0E026FDECF10F0DDCF11F0FF0E101A51
:10126000111A10C0DEFF11C0DDFFDF2A010E01E3FD
:10127000DB2ADECF10F0DDCF11F00A0E1102F3CF22
:1012800011F01002F3CF10F0F4501126040ED89094
:1012900011321032E804FBE110C0DEFF11C0DDFFA7
:1012A000040EF36E020EF3CFDBFFDB50000833E2D7
:1012B000DECF10F0DDCF11F00A0E0B6E0C6A10C0FD
:1012C00006F011C007F04FEC0CF002C010F003C0A4
:1012D00011F00F0E10143009E66E020EDB50EA6AB0
:1012E000020FE96E010EEA22E552E750EF6ED9CF08
:1012F000E9FFDACFEAFF0A0E0B6E0C6AEECF06F0BA
:10130000EDCF07F04FEC0CF006C0EEFF07C0EDFF8D
:10131000020EDB06CAD7300E0101035D07E1200E85
:10132000036F300E045D02E1200E046F06C107F169
:101330002E0E066FF80E086F430E096F0D0E0A6F22
:101340000B6B030EE15C02E2E16AE552E16EE552ED
:10135000E7CFD9FF120080A203D06DA60FD802D02C
:101360006DB613D801011E0508E16DBA06D0686A92
:10137000696A69806988020E1E6F12006D6A696A67
:101380006D860101010E1E6F12006D6A696A01010E
:101390001E6B1200C5EF09F001011E5101E13AD0A8
:1013A0006850040B04E06950040B01E03CD86DB2B6
:1013B00031D06850010B04E06950010B01E054D8B2
:1013C0006850100B04E06950100B01E024D86850FD
:1013D000400B04E06950400B01E03BD86850200B03
:1013E00004E06950200B01E036D86850020B04E09D
:1013F0006950020B01E036D8030E01011E5D01E2C7
:1014000009D06850080B06E06950080B03E05FEC58
:1014100007F068961200698468986D82A19AA08A84
:101420000300A09A12006D92699468941200010161
:101430001FA10ED0F8DF6D840001080EFD6F070EAE
:10144000FE6FFD07000EFE5BFD51FE11FAE16D948B
:101450001200689C120070A003D0CEEC08F07090CF
:10146000689A1200689212006A6A686A9F0E6B6E30
:101470007B0E696E6E6A0F0EE66E710EE66E0F0ED3
:10148000E66E14D8E552E552E552160E706E68A667
:1014900002D06896FCD76D98CEEC08F001011F9140
:1014A0000101206B0101030E1E6F1200D9CFE6FF70
:1014B000E1CFD9FFFD0EDBCFE9FFFE0EDBCFEAFF68
:1014C000FC0EDB5004E0EE6AFC0EDB06F9D7E552B9
:1014D000E7CFD9FF1200F00E8C1695169388938AE9
:1014E0008150100B01E0010E0001606F8150200B54
:1014F00001E0010E616FDCEC08F07FEF0AF0948EE2
:10150000949C710EAF6E020EB06E240EAC6E900EF7
:10151000AB6E080EB86E120023D8060E01011E5DD8
:1015200003E36D50020B01E006D006D814D814D89E
:1015300014D814D814D812005BD800090BE00001AD
:10154000E35108E10E0EE66E180EE66E23EC05F090
:10155000E552E552120012001200120012001200B1
:1015600001012251231104E1100E226F270E236F77
:101570002207000E235B6DA20BD02251231107E13D
:101580008C708C50010B02E08C8201D08C922FD099
:1015900001011E5103E18C908C9229D01E0503E1BC
:1015A0008C808C8224D0020E1E5D03E18C808C9294
:1015B0001ED0030E1E5D03E18C908C8218D0050EA8
:1015C0001E5D07E101012251231102E18C708C9212
:1015D0000ED0060E1E5D0BE101012251231107E121
:1015E0008C708C50010B02E08C9201D08C82120026
:1015F0008150100B01E0010E0001605D09E0815097
:10160000100B01E0010E606F81B802D0010E02D014
:10161000000E00D012008150200B01E0010E0001ED
:10162000615D09E08150200B01E0010E616F81BA1C
:1016300002D0010E02D0000E00D0120012010002F2
:1016400002000008D8040A0000000102000109029B
:10165000430002010080320904000001020201007F
:1016600005240010010424020205240600010524BB
:101670000100010705820308000209040100020AB3
:101680000000000705030240000007058302400038
:10169000000403090434034D006900630072006F05
:1016A000006300680069007000200054006500635A
:1016B0000068006E006F006C006F0067007900200A
:1016C0000049006E0063002E0034034300440043D1
:1016D000002000520053002D003200330032002061
:1016E0000045006D0075006C006100740069006FBA
:1016F000006E002000440065006D006F004E164E25
:101700001691169516C9163808FF2A0EF66E080EA1
:10171000F76E000EF86E01010900F550116F090017
:10172000F550126F03E1116701D03DD00900F5506B
:101730000C6F0900F5500D6F0900F5500E6F090090
:101740000900F550E96E0900F550EA6E090009003C
:101750000900F5500F6F0900F550106F09000900DE
:10176000F6CF13F1F7CF14F1F8CF15F10CC1F6FF56
:101770000DC1F7FF0EC1F8FF01010F5302E1105335
:1017800007E00900F550EE6E0F07F8E21007F9D7F1
:1017900013C1F6FF14C1F7FF15C1F8FF01011107CE
:1017A000000E125BBFD71200D9CFE6FFDACFE6FFFB
:1017B000E1CFD9FFE2CFDAFF3F0EC716C66AFD0EB2
:1017C000DB50C612FB0EDB50C712FC0EDB50030AC7
:1017D00009E0010A04E0020A06E1C78C04D0C78CC4
:1017E000C68801D0C688FD0EDB50050A03E0010A59
:1017F00004E1928A9382C79E01D09392949E938033
:10180000C68AE552E5CFDAFFE7CFD9FF120050498B
:1018100043313846343535302046756C6C2D537065
:1018200065656420555342202D2043444320525384
:101830002D32333220456D756C6174696F6E2044B2
:10184000656D6F0D0A0D0A001B5B324A00547970FA
:101850006520696E206120737472696E6720686507
:1018600072652E0D0A0005D812D88CEC0AF0FCD750
:1018700012000F0EC11292829284140E6F6E01013B
:101880001E6B01011F6B0101206B6BEF0AF0ABECCB
:1018900009F06FBE02D0CCEC09F061EF05F0036AED
:1018A000026A100EE76ED890063607360236033607
:1018B0000B50025C0C50035805E30B50025E0C50B9
:1018C000035A062AE72EF0D7120013EE00F023EE9B
:1018D00000F0F86A0F9C85EC0BF033EC0CF0FDD7B0
:1018E0001200C96AC7A0FED7C95012000000FFFF4E
:0200000400F00A
:10000000FFFFFFFFFFFFFFFFFFFFFFFFFFFFFFFF00
:10001000FFFFFFFFFFFFFFFFFFFFFFFFFFFFFFFFF0
:10002000FFFFFFFFFFFFFFFFFFFFFFFFFFFFFFFFE0
:10003000FFFFFFFFFFFFFFFFFFFFFFFFFFFFFFFFD0
:10004000FFFFFFFFFFFFFFFFFFFFFFFFFFFFFFFFC0
:10005000FFFFFFFFFFFFFFFFFFFFFFFFFFFFFFFFB0
:10006000FFFFFFFFFFFFFFFFFFFFFFFFFFFFFFFFA0
:10007000FFFFFFFFFFFFFFFFFFFFFFFFFFFFFFFF90
:10008000FFFFFFFFFFFFFFFFFFFFFFFFFFFFFFFF80
:10009000FFFFFFFFFFFFFFFFFFFFFFFFFFFFFFFF70
:1000A000FFFFFFFFFFFFFFFFFFFFFFFFFFFFFFFF60
:1000B000FFFFFFFFFFFFFFFFFFFFFFFFFFFFFFFF50
:1000C000FFFFFFFFFFFFFFFFFFFFFFFFFFFFFFFF40
:1000D000FFFFFFFFFFFFFFFFFFFFFFFFFFFFFFFF30
:1000E000FFFFFFFFFFFFFFFFFFFFFFFFFFFFFFFF20
:1000F000FFFFFFFFFFFFFFFFFFFFFFFFFFFFFFFF10
:020000040030CA
:0E000000240E3F1E008181000FC00FA00F4094
:020000040020DA
:08000000FFFFFFFFFFFFFFFF00
:00000001FF
